:10000000982AFF3FFF3FFF3FFE0003088301D70010
:100010007F08D60083010C1C2D2883160C1C2D286C
:1000200083120313101083160C1083120C10AC01F2
:10003000A1100B12831601138B100B1683122017BD
:100040002308043A031D2C2803302A0203182C2805
:100050000430AE00A0162D28A5018B180B1E552AC2
:100060008312031310100F08CE00CD010E08CF002D
:10007000D0014D08CF070318D00A4E08D007003032
:100080004F07CB003830031839305007CC0003102D
:10009000CB0DCC0D0310CB0DCC0D4C08A4001010D3
:1000A0008E01C8308F000C10101483160C148B10A6
:1000B000332A0130AC0083160117552A0230AC00F8
:1000C0008316011383122408A700A01B552A831648
:1000D0002B0883122702031C7228270883162C0280
:1000E000031874288312B12883122308A900552A03
:1000F0008316011704308312AC00AA01B101B201CA
:10010000B301B401AE012408A600A01F8928A016DF
:10011000552AA01283162D0883122602031C952847
:10012000260883162E020318BE2883122308053AD8
:10013000031DB128031083162D0C83122602031C05
:10014000B128031083162E0C03138312CD0026084A
:100150004D02031CB1280830A900A8000130AE00F0
:10016000242A101083160C1083120C10AC01A1105D
:100170000B12831601138B100B16552A83122308BA
:10018000A8002803031D552AA110552A8316011320
:1001900083122408A7000330AC00280B552A24083A
:1001A000A600AE01DD28AE018316011783122408D4
:1001B000A6000430AC00280B292906302602153091
:1001C000031CE82826020318E728A701F4281530A5
:1001D0002602031CF228233026020318F2280130DD
:1001E000A700F4280330AE002E08033A031DFC28B4
:1001F0002A080C3A031D242A270803190129A110F3
:1002000003290230A106A11C09298316011F0C290C
:100210000F298316011F0F2983122114112983121C
:10022000211083120313A11C182927080319552A2A
:10023000003021180130B1040C30AA0A2A02031838
:1002400027290310B10DB20DB30DB40D552A01309D
:10025000212A2808043A031935292808053A0319E0
:1002600035292808023A031D9D292808023A031D52
:100270003B290B303C292030AB00A11083162F08FE
:1002800083122702031C582927088316300283167D
:10029000031C5929310883122602031C5829831292
:1002A000260883163202031C58298312A1147229CE
:1002B0008316330883122702031C6F29270883162D
:1002C0003402031C6F298316350883122602031C8F
:1002D0006F29831226088316360203187229033009
:1002E0008312AE008312A11C7729311478293110B2
:1002F0002E08033A031D80292A082B06031D242AF1
:100300002B08CD00CE01FF30CD07031CCE072A08F5
:10031000CF00D0015008803AFF004E08803A7F029B
:10032000031D94294D084F0203189D2903108312C1
:100330000313B10DB20DB30DB40D831203132808CE
:10034000033A031D042A3030AB00A11083162F0896
:1003500083122702031CC029270883163002831644
:10036000031CC129310883122602031CC0298312F1
:10037000260883163202031CC0298312A114DA292D
:100380008316330883122702031CD72927088316F4
:100390003402031CD7298316350883122602031C56
:1003A000D72983122608831636020318DA29033068
:1003B0008312AE0083122E08033A031DE3292A0894
:1003C0002B06031D242A20302A020318F629A11C1B
:1003D000EB293114EC2931101F302A020318042AAA
:1003E0000310B10DB20DB30DB40D042AA11CFA29EE
:1003F0002F14FB292F102F302A020318032A031071
:10040000AF0DB00D042A64002B08CD00CE01FF30E3
:10041000CD07031CCE072A08CF00D0015008803A30
:10042000FF004E08803A7F02031D182A4D084F0234
:1004300003181E2A83120313AA0A552A01308312B5
:100440000313AE000530AC00A016101083160C107C
:1004500083120C10AC01A1100B12831601138B1028
:100460000B160B12552A83122C08003A031959282F
:10047000013A03195E28033A03197828013A03194F
:10048000D328073A0319C628013A0319242A101061
:1004900083160C1083120C10AC01A1100B128316E2
:1004A00001138B100B168312A0128B1A0B1D8F2AAF
:1004B0000B11813083120313810083162608031D5C
:1004C000A6032708031DA703A50A2508643A031DF0
:1004D0008F2AA501220803196E2AA2032308031DEF
:1004E000A303A10A21080A3A031D8F2AA1012A08A1
:1004F00003197B2AAA03A90A29080A3A031D852A97
:10050000A90124080319852AA403A80A2808783A0F
:10051000031D8F2AA80183125108031DD103031361
:1005200083125608FF0057088300FE0E7E0E090056
:10053000531083195314D310031AD314203084009A
:100540005130AA22A0308400B730AA22C52A04065E
:100550008001840A0406031DA72A64000034831264
:100560000313D400D51BBD2A551BC52A55088A0084
:100570005408D40A0319D50A820083135518831727
:100580005408D40A840000080800831603138E1C44
:10059000031ECE2A8312D20183160E140E18D22AFD
:1005A0008312D20183168E140E14D326520BDD2A29
:1005B00086158B172926BC25E12A9B272926A024EE
:1005C0002926A2278B176400D723BC00831627088F
:1005D00083120319BC080319A501BC080319F32AE7
:1005E000C8308316A7008312BD01032B66270D2B8D
:1005F000831623088312031D0E2B2D0B002B0D2BAE
:100600002D08BD000D2B3C08013A0319F62A033AC8
:100610000319002B013A0319F82A8312BD080319A4
:10062000CA2B3D08BE00BF013F08073ED5003E086B
:10063000893E0318D50AAF228316A300CA2B9B2735
:10064000851E242B3D0BE32AD201D20A86151030D9
:100650009227B900B908031D2F2BB901B90ABC258F
:10066000061186101430C62B8615831626088312B1
:10067000031D3C2B861006113D08023A031D482B32
:100680008614831620088312D1003B088316A60027
:1006900083123D08033A031D552B061583162008C7
:1006A0008312D1003B088316A6008312851E622B9D
:1006B0003D0B5B2B622B5108031D6B2B8316A0088F
:1006C00003196B2B8312B901BC2506152208792763
:1006D00006119B27E32A831220188A2B061A732BF4
:1006E000B901B90ABC25861A782B0230B900BC259D
:1006F00003303A02031C952B061B812B0330B900F3
:10070000BC2504303A020318861B952B0430B9002F
:10071000BC25952B061A952B3A083902031C912B00
:10072000B901B90ABC25023079273D08043AA0185E
:10073000BC2B031D9E2BB901B90ABC253D08053A07
:10074000031DA52B0230B900BC2503303A02031C5F
:10075000E32A3D08063A031DB02B0330B900BC253F
:1007600004303A02031CE32A3D08073A031DE32A3A
:100770000430B900BC25E32A031DE32A3A083902F4
:10078000031CC32BB901B90ABC2502307927E32A1F
:10079000D201E32A83125208003A03191F2B013AAF
:1007A0000319342B033A0319C82B013AC82B8301D0
:1007B000AD01230803190034A01E201BE02B0034D8
:1007C0002308043A0319EB2B201BE92B2E030319F2
:1007D000F92B662700342E08043A031DF92BA508CF
:1007E0000319F72B20162508AD006627033466276A
:1007F00000342808083A031D062C2308053A031D77
:10080000062C20162508AD0066270334B501B60175
:10081000B701B8013A2CFF303105B5000730320579
:10082000B600B21D152C20154A2C20114A2C310877
:10083000B5003208222C3108B7003208B8002F0862
:10084000B5003008B6004A2C201B292C2E030319B2
:10085000312C662700342808083A031D312C6627FE
:1008600000343108B5003208B6003308B700340848
:10087000B8004A2C2308013A03190B2C033A031938
:10088000172C013A03191B2C073A0319242C013A9F
:1008900003192B2C8312031338083704360435044C
:1008A000031D542C6627003420122030C700C601D7
:1008B000470892273806031D702C470A92273706EF
:1008C000031D702C4708023E92273606031D702C2C
:1008D0004708033E92273506031D702C2016772CFF
:1008E000C60A0430C70707304602031C582C201ED6
:1008F0009D2C460AAD006627230B962C201D822CCA
:100900000130832C0030C800A01D882C0130892CB8
:100910000030C806031D902C25082D06031903344A
:10092000A0112019A0152D08A500023425082D06B8
:10093000031903342D08A50002346627AD010134E4
:100940008301061A0800061E861AAB2C83018B173A
:1009500005303C274D2E8B1703303C274D262308AE
:10096000C400A30185152308031DCB2CA301A227D6
:10097000C201C301C208031DC12C4025C20064008E
:10098000BA2C2808A3002308073985004D261E30FD
:1009900079278501B32C01303C27A227C401C0016F
:1009A000C1012030C300051464008312C10803197B
:1009B000FF2CC10138083704360435040319FE2C16
:1009C000430892273806031DF82C430A922737065E
:1009D000031DF82C4308023E92273606031DF82C0F
:1009E0004308033E92273506031DF82C2627FF2CCB
:1009F000AD080319FE2C2D0A3C27FF2C1027851A61
:100A0000282D262703307927C0080319102D440A02
:100A10003C2744089126C00103307927C101112DDC
:100A200010270730C40A4402031C1A2D640026272D
:100A30001027162D4408C5000310C50D0310450DE1
:100A4000203EC300B501B601B701B8014D2605141B
:100A500083162708031DD42CD723C200420B312D47
:100A6000352D4208023A031DD42CC8308316A70046
:100A70008312C101C10AC001C00AA5010510D42C0E
:100A8000640083120313A017A01E00340B12101071
:100A9000A90106302702031C5B2D1530270203181D
:100AA0005B2D06302602031C5B2D15302602031831
:100AB0005B2D0130B42D1F302702031C6D2D2F300C
:100AC000270203186D2D05302602031C6D2D0B30F7
:100AD000260203186D2D0230B42D2E302702031C80
:100AE0007F2D3F30270203187F2D15302602031C6F
:100AF0007F2D1D30260203187F2D0330B42D3B308F
:100B00002702031C912D513027020318912D3B30F1
:100B10002602031C912D513026020318912D04301A
:100B2000B42D77302702031CA32DA230270203180F
:100B3000A32D3B302602031CA32D5130260203189F
:100B4000A32D0530B42D77302702031CB52DA2301C
:100B500027020318B52D1D302602031CB52D2930A0
:100B600026020318B52D0830A9002908A8000B1289
:100B7000A012A301A2270134830139083A02031805
:100B8000C32D3A08B9000510851005118511E12D16
:100B900085130513F12D851305130514F12D851308
:100BA00005178514F12D04303A02031CD92D0513C5
:100BB000DA2D051785170515F12D851705178515EC
:100BC000F12D3908003A0319C82D013A0319CB2D2C
:100BD000033A0319CF2D013A0319D32D073A03190C
:100BE000DD2DB908031908001030C9003908F326B3
:100BF000831620088312D1000230792FFF3FFF3F78
:100C0000820706341434153422340634143415346F
:100C100022340F34153405340C3405340C340534C7
:100C20000C3404340A340F34163404340A340334D4
:100C3000093404340C3413341B3404340C340434B9
:100C40000C3406340B3415341B3406340B340634A0
:100C50000B3410309227B90009309227BA000830BF
:100C600092278316A00013309227A3000A30922700
:100C7000003803193D2E20143E2E20100B309227F1
:100C800000380319452EA014462EA0100C309227D0
:100C9000BB000D309227A2000800830121156C2EA5
:100CA0006400851A061E592E861A061F592E861BA9
:100CB0005B2E21155C2E21110230792721196C2E13
:100CC000851A061E692E861E692E061B861F692E32
:100CD0006B2E21156C2E2111211D0800502E830131
:100CE000C600C7014708AF3E84008313C608031936
:100CF000872E06308A004608C8000310C80D03106E
:100D0000C80D0310480D4707F83E0026882E003016
:100D1000800083120313C70A083047020318080033
:100D2000722E8301C600C608031D9A2E1330C90017
:100D30002308F3264608C8000310C80D0310480D09
:100D4000203EC700C9003808F326470AC900370803
:100D5000F3264708023EC9003608F3264708033E3B
:100D6000C9003508F32E8301C600C7014708AB3E12
:100D700084008313C6080319C92E07308A00460869
:100D8000C8000310C80D0310480D4707FC3E51274B
:100D9000CA2E0030800083120313C70A04304702B2
:100DA00003180800B62E83018501860107309F00D5
:100DB00083169F0183129813970183168E15203096
:100DC0008500F13086000230810020308B008130B8
:100DD000831281009001013092009101831601136A
:100DE0000B17831208008301CA00490883169B0071
:100DF00083124A0883169A0003108B1B03148B136B
:100E00001C1555309D00AA309D009C141C11031820
:100E10008B179C1C0D2F6400092F9B018312080067
:100E200083010510851005118511051401307927FE
:100E300005108514013079278510051501307927B3
:100E400005118515013079278511080083010510EA
:100E50008510051185118515013079278511051536
:100E60000130792705118514013079278510051483
:100E700001307927051008008301C600C700C708A4
:100E80000319080005148514051585150330792705
:100E9000051085100511851103307927C70B422FE6
:100EA0000800820706341434063414341F342E34F8
:100EB00005340A342E343E3415341C343B3450345B
:100EC0003B3450347734A1343B3450348301A01286
:100ED0002013A013AA01101083160C1083120C10FB
:100EE000AC01A1100B12831601138B100B16831289
:100EF00008008301C800C8080319862F4808831614
:100F0000A20022080319862F6400812F8312080093
:100F1000820701343234013401341E341E341E344D
:100F20001E3401348301C90083169B009C131C14DA
:100F30001A08831208008301D20186110611861057
:100F4000B901BC2D83012308B32623086F26662F21
:100F500083010800FF3FFF3FFF3FFF3FFF3FFF3F91
:100F6000FF3FFF3FFF3FFF3FFF3FFF3FFF3FFF3F91
:100F7000FF3FFF3FFF3FFF3FFF3FFF3FFF3FFF3F81
:100F8000FF3FFF3FFF3FFF3FFF3FFF3FFF3FFF3F71
:100F9000FF3FFF3FFF3FFF3FFF3FFF3FFF3FFF3F61
:100FA000FF3FFF3FFF3FFF3FFF3FFF3FFF3FFF3F51
:100FB000FF3FFF3FFF3FFF3FFF3FFF3FFF3FFF3F41
:100FC000FF3FFF3FFF3FFF3FFF3FFF3FFF3FFF3F31
:100FD000FF3FFF3FFF3FFF3FFF3FFF3FFF3FFF3F21
:100FE000FF3FFF3FFF3FFF3FFF3FFF3FFF3FFF3F11
:100FF000FF3FFF3FFF3FFF3FFF3FFF3FFF3FFF3F01
:084000000A00010002000100AA
:02400E00543F1D
:10420000330000000000000000000000000000007B
:10421000B40004000000010064000000100005006C
:10422000010020004000030000000000000000002A
:104230004A0041005000360020004900520043006F
:1042400009000000BC00B50009000000C000C90062
:10425000090000004000490009000000300039005A
:10426000090000000000090009000000600069006A
:10427000FA005500AF00AA00FF005500FF00FF0044
:10428000FA005500AF00AA00FF005500FF00FF0034
:10429000FA005500AF00AA00FF005500FF00FF0024
:1042A000FA005500AF00AA00FF005500FF00FF0014
:1042B000FA005500AF00AA00FF005500FF00FF0004
:1042C000FA005500AF00AA00FF005500FF00FF00F4
:1042D000FA005500AF00AA00FF005500FF00FF00E4
:1042E000FA005500AF00AA00FF005500FF00FF00D4
:1042F000FA005500AF00AA00FF005500FF00FF00C4
:00000001FF
